:020000000B28CB
:10000800DF0003088312A0000A08A1003128831624
:10001800FF239000830157284C2041208B16241C75
:100028001328051C851C2C280130230222300319B3
:100038002202031C212805112F2800302302283012
:100048000319220203180515A20A0319A30A2F2867
:100058000511A201A3012410132885168B1A0B1D64
:100068003928EB30810024140B11851221088A00ED
:1000780020088300DF0E5F0E0900810183168111BD
:10008800011181100114811283128B128B17080041
:100098000730990083169F01811795010511851274
:1000A800831285010800A401A201A301830110287D
:02400E00E43F8D
:00000001FF
